:06000000008074022B9247
:03000B0002215679
:0300130002203692
:03001B0002225E60
:03002300022B3B72
:10002B0032534D505445204D616368696E652020F5
:10003B00202863292031393936202020416C636F09
:10004B00726E204D63427269646520496E632E2087
:10005B0020200D534D505445204D616368696E65EA
:10006B00202020012056312E36390D00C2AF75D01D
:10007B000075816B43B0FF4390FF75892175880430
:10008B00758DFD758BFDD28E7589237598D0787F14
:10009B00E4F6D8FD751800751E149000007400F07E
:1000AB00A3A883B820F974FF90E800F0901523F013
:1000BB0090E000F0901522F090E000E0F890E8005E
:1000CB00E05875A015781EF2D294D2961201769054
:1000DB002D2112022A902D3412022A122CB8121A38
:1000EB00DD121AB5121E8C122CC6122CB8121EF170
:1000FB00122CB8122CB8122CB8C294122CC6D29453
:10010B0075B80075A811D2AF751296D221C215C25F
:10011B003FD201302A02C20175816B300144C28C7F
:10012B00758A00754C00C204D246D28CD2A9902D90
:10013B002112022A902D3412022AC22712050430F2
:10014B002303120BB93001121202C73004EEC204A2
:10015B00B2941207DB30010280E2C28CC2A9C24604
:10016B00D2922022030214B302170F90000075A045
:10017B00A07802E230E70BA3E583B405F6C23802A0
:10018B0001C7D2387A301201C87A301201C87A38D6
:10019B001201C87A801201C87A061201C87A0C12B1
:1001AB0001C87A011201C87A401201C87A5A1201A9
:1001BB00E77A401201C8120209B45AC122C0F030CA
:1001CB00381775F00075A0A07802E230E70700D56C
:1001DB00F0F30201E47800EAF2D0F022C0F03038FC
:1001EB001A75F00075A0A07802E230E70700D5F091
:1001FB00F302020675A0A07801EAF2D0F022C0F05B
:10020B0030381975F00075A0A07802E230E70700CE
:10021B00D5F0F302022775A0A07803E2D0F0227488
:10022B000093A3120248FA740093A32AFA1201C88E
:10023B00740093A36006FA1201E780F42283227FF5
:10024B00BF93D37A851201C8E55175F00060047530
:10025B00F00A842430FA1201E7E5F02430FA120197
:10026B00E77A3A1201E7E55275F000600475F00A7F
:10027B00842430FA1201E7E5F02430FA1201E77A10
:10028B003A1201E7E55375F000600475F00A842417
:10029B0030FA1201E7E5F02430FA1201E77A2E1258
:1002AB0001E7E55475F000600475F00A842430FA18
:1002BB001201E7E5F02430FA1201E722303A08E5A3
:1002CB006830E0031202EB303B08E56830E10312C3
:1002DB000422303C08E56830E203120425C23A22BE
:1002EB00E562C39561F4B412005003020421A862C5
:1002FB0075A01C74FEF2F5F075A01B7401F2087565
:10030B00A01CE56AF225F0F5F075A01BE4F2087568
:10031B00A01C7428F225F0F5F075A01BE4F208750B
:10032B00A01CE569F225F0F5F075A01BE4F2087549
:10033B00A01CE551F225F0F5F075A01BE4F2087551
:10034B00A01CE5F0C313F275A01B7401F20875A095
:10035B001C74FEF2F5F075A01B7401F20875A01C5D
:10036B00E56AF225F0F5F075A01BE4F20875A01C08
:10037B007428F225F0F5F075A01BE4F20875A01CAB
:10038B00E5692401F225F0F5F075A01BE4F2087580
:10039B00A01CE552F225F0F5F075A01BE4F20875F0
:1003AB00A01CE5F0C313F275A01B7401F20875A035
:1003BB001C74FEF2F5F075A01B7401F20875A01CFD
:1003CB00E56AF225F0F5F075A01BE4F20875A01CA8
:1003DB007428F225F0F5F075A01BE4F20875A01C4B
:1003EB00E5692402F225F0F5F075A01BE4F208751F
:1003FB00A01CE553F225F0F5F075A01BE4F208758F
:10040B00A01CE5F0C313F275A01B7401F2088862FF
:10041B009060057406F022C23B22E562C39561F43D
:10042B00B40C005003020503A86275A01C74FEF205
:10043B00F5F075A01B7401F20875A01CE56AF22596
:10044B00F0F5F075A01BE4F20875A01C7428F225DA
:10045B00F0F5F075A01BE4F20875A01CE569240407
:10046B00F225F0F5F075A01BE4F20875A01C9015B1
:10047B0063E0F225F0F5F075A01BE4F20875A01C03
:10048B00E5F0C313F275A01B7401F20875A01C7480
:10049B00FEF2F5F075A01B7401F20875A01CE56A5D
:1004AB00F225F0F5F075A01BE4F20875A01C74287A
:1004BB00F225F0F5F075A01BE4F20875A01CE569B8
:1004CB002405F225F0F5F075A01BE4F20875A01CCD
:1004DB00901564E0F225F0F5F075A01BE4F20875B9
:1004EB00A01CE5F0C313F275A01B7401F20888621F
:1004FB009060057406F0C23C22E559655A600812FB
:10050B00053220232180F2E563656460081206D86A
:10051B0020231380F2E55F6560600B202D05120729
:10052B002C80031226BA2220210302060175A01E7D
:10053B00A959E3FA75A01DE3FB0559C239C229BBC2
:10054B000006EA20280F802BEA30E72590155CF097
:10055B00D228020600C228B4FE0DF51CF51D751835
:10056B0000751E14020600B480005015751D008026
:10057B0047D229AD1DBDFE0302058FBD0003020549
:10058B00DF020600BB0002801AF5F090155CE02537
:10059B001CC313B5F005D223020600745512148840
:1005AB00020600851EA0A818F2251CF51C08881849
:1005BB00B80002051E02060090155CE075831C85D1
:1005CB006282F0740175831BF00582E561658260C0
:1005DB002485826220391E75831C856282EAF0EBCA
:1005EB0075831BF00582E5616582600985826290E7
:1005FB0060057406F02275A01EA959E3FA0559C2CD
:10060B0039C229BAF50CEA202816201D31201C39D5
:10061B008044EA90155CF0C21DC21CD2280206D79A
:10062B00C228D21DB4FE0DF51CF51D751800751EE4
:10063B00140206D7B48000502B751D00805CC21DC0
:10064B00D21C251CF51C0206D7C21CFB0B251CF566
:10065B001C0206D7D229AD1DBDFE0302058FBD00BE
:10066B00030206BB0206D71BBB001AF5F090155C04
:10067B00E0251CC313B5F005D2230206D77455121F
:10068B0014880206D7851EA0A818F2251CF51C0895
:10069B008818B80002051E0206D790155CE075831A
:1006AB001C856282F00582E5616582601F8582622E
:1006BB0020391975831C856282EAF00582E5616534
:1006CB008260098582629060057406F02230212BCE
:1006DB0075A01AA963E3FA75A019E3FB056375838B
:1006EB001F855C82EAF00582E55B6582600385828B
:1006FB005C202002D299D23902054875A01AA96351
:10070B00E3FA056375831F855C82EAF00582E55B7E
:10071B006582600385825C202002D299D239020661
:10072B000C75A016A85FE2055FB4FE0BD230C23188
:10073B00C232C2330207DA30300AB41302D231C2EA
:10074B00300207DA303110B42000505E901563F0A0
:10075B00C231D2320207DA30320A901564F0C2325B
:10076B00D233806B30334BF87A11901563E02AFA51
:10077B00901564E02A547FC398702F901564E0F8AD
:10078B00901563E09015652582F58274003583F52D
:10079B0083E8F0D23C30E504D234800375661E90BA
:1007AB001522E054FDF090E000F0C231C232C233AA
:1007BB00801DC231C232C23375831F855C82F00546
:1007CB0082E55B6582600385825C202002D29922E0
:1007DB0090E800E0F890E000E058C0E075A01578D4
:1007EB001EE2FAD0E0F26A5AFAEA541F604D30E08A
:1007FB0025D291C201201510200015C23F302210C6
:10080B00301F0D1219388008103F0280031219385F
:10081B00C200C215802530E105202B02D20030E347
:10082B0004D201801630220E30E402D21530E20BD6
:10083B00D201D291800530E202D201227851E60832
:10084B00460846084660121208657002800B1208B3
:10085B00F260067D16DDFE80F522900000E060263A
:10086B00F975650030257D20267A7E107F008E82FB
:10087B008F83E0B4FF02806CF5F07851E6B5F0029F
:10088B0080104060D902805C74082EFEEF3400FFAC
:10089B0080DCA3E0B4FF02804BF5F008E6B5F00274
:1008AB008004404080DEA3E0B4FF028037F5F008FF
:1008BB00E6B5F0028004402C80CAA3E0B4FF0280AE
:1008CB0023F5F008E6B5F0028004401880B6E56524
:1008DB00B4000DA3AB82AC83901520EBF0A3ECF02E
:1008EB00056580A0E56522901520E0FBA3E0FCE503
:1008FB0065B400030209398B828C83E0FEA3E0FF11
:10090B00A3E0F97003020928A3E0B4FF0302093C3A
:10091B00B48000500302096BD565028011EB2408EB
:10092B00FB901520F0A3EC3400FCF0020902E56506
:10093B0022E55CC3955BF489F0B5F0005003020926
:10094B00398E828F83A85C75A01FE0F2A308D9FAB9
:10095B00885C202002D299D5650302093902092847
:10096B00E562C39561F489F0B5F0005003020939D3
:10097B008E828F83A86275A01CE0D2E7F275A01B54
:10098B007401F2D903088022A308D902800FE07505
:10099B00A01CF275A01B7400F2A308D9F1E075A09E
:1009AB001CF275A01B7401F2A30888629060057499
:1009BB0006F0D56503020939020928E538C4540F3E
:1009CB00F5F0E53954F045F030E72530E622543F99
:1009DB00F5F0B43F028024900007E0B5F002801BD5
:1009EB00901500E0600AFAA3E0B5F002800DDAF78B
:1009FB0090153EE4F0A3F0A3F08008901536E5F0D7
:100A0B00F0D21622901536E0F5F0A3E53AC4540F58
:100A1B00F9E53B543049F025F0F5F0A3E53CC4541F
:100A2B000FF9E53D543049F025F0543FF5F09015A2
:100A3B0036E5F0F022901536E0F5F0E53EC4540FA4
:100A4B00F9E53F543049B5F002800B90153EE4F0C8
:100A5B00A3F0A3F08020C21E7903783E75A015E2A7
:100A6B00F5F0E0B5F0028002D21EF2121D39D9EF7B
:100A7B00301E03021D41227400B5520DB5530AB549
:100A8B0051077403B55400500122901526E060F90C
:100A9B00FA7400F0A3A85E121E85B4030040F8752B
:100AAB00A018E0D2E7F2FB75A0177401F20875A04D
:100ABB00187408F22BFB75A0177400F20875A018B8
:100ACB00EBF275A0177400F208885E75A0807905AB
:100ADB007406F3A3DAC1C21B22900000E07005D2AA
:100AEB0026020B3D75F000900005E0C395F09000D9
:100AFB0003F075F008900006E095F0900004F0907C
:100B0B000000E0C226C394025002802604FA750549
:100B1B00137504008504068505077907120BAFEAE8
:100B2B00FB120B407907120BAFDBF67905120BAFFB
:100B3B00DAE2D22522C082C083A8058504A08507EE
:100B4B0082850683E0F5F0E2C395F0C0D0120B87E7
:100B5B00E0F5F0E2D0D095F0C0D0120B87E0F5F0C5
:100B6B00E2D0D095F0C0D0120B87E0F5F0E2D0D0F8
:100B7B0095F04003120B9BD083D08222C0E01582EC
:100B8B00E582B4FF02158318B8FF0215A0D0E0224E
:100B9B007908E2F5F0E0F2E5F0F0A308B800020501
:100BAB00A0D9EF22E72408F719E73400F7229014B5
:100BBB0000E0B44203020E01543F2323900BCB738E
:100BCB00020CD300020EF100020F9200020FA300E1
:100BDB00020FC000020CCB00020FCE00020FF4007C
:100BEB0002102E000210BC00021290000212B40080
:100BFB000212DA000212F40002130000021350007A
:100C0B000213A7000214800002145C0002143600C9
:100C1B0002140D0002104D0002106D000212240090
:100C2B000213320002133F00020CCB00020CCB006C
:100C3B00020CCB00020CCB00020CCB00020CCB0045
:100C4B00020CCB00020CCB00020CCB00020CCB0035
:100C5B00020CCB00020CCB00020CCB00020CCB0025
:100C6B00020CCB00020CCB00020CCB00020CCB0015
:100C7B00020CCB00020CCB00020CCB00020CCB0005
:100C8B00020CCB00020CCB00020CCB00020CCB00F5
:100C9B00020CCB00020CCB00020CCB00020CCB00E5
:100CAB00020CCB00020CCB00020CCB00020CCB00D5
:100CBB00020CCB00020CCB00020CCB00020CCB00C5
:100CCB007455121488C22322901401E0B4FE03025F
:100CDB000CF7B4FF03020D25B40003020D25B4FD80
:100CEB0003020D257455121488C22322120D0274AF
:100CFB00AA121488C223227A079000007400F0A372
:100D0B00DAFCD226D225751800751E14751F0074D7
:100D1B0000900005F07408A3F022C21EF5F0202607
:100D2B0006900000E07003020DF0FBF51F7A01A99D
:100D3B00F0EA75F008A4240FF582E5F03400F58392
:100D4B0089F0E0B5F0028003020DE3D21EE582C309
:100D5B009403F582E5839400F583E0FCA3E0FDA307
:100D6B00E0F9E51FC39A04C0F075F008A4AFF0FEDC
:100D7B00EA1475F008A42410F8E5F03400F5A0EAA5
:100D8B0075F008A42410F582E5F03400F583120EFB
:100D9B002CECF8EDF5A0E92CF58274003DF583748D
:100DAB0000C39582FE74149583FF120E2C900003E2
:100DBB00E0C399F0A3E09400F0A3E0C399F0A3E0A3
:100DCB009400F0120E3BD0F01B151FE51FB400036F
:100DDB00020CF7BB000C800D0ABB00028007DB0284
:100DEB008003020D3A301E06E51F900000F074AA36
:100DFB00121488C22322A85C90005E7900E99360EC
:100E0B0016B40102744175A01FF20908E8B55BED39
:100E1B002020FAD29980F6885C202002D299C22336
:100E2B0022E0F2121D39DEF9BF00028002DFF2224E
:100E3B00900014E51F6029F8E0C39CAE82AF83A33A
:100E4B00E09505400D8E828F83E0C399F0A3E0946B
:100E5B0000F074072582F58274003583F583D8D8AA
:100E6B0022900000E0F5F0FA7B007E0D900003E08D
:100E7B002AFA74003BFBA3DEF6900010AEF0BE0026
:100E8B0003020E9D7F08E02AFA74003BFBA3DFF6FA
:100E9B00DEF2900003E0FFA3E0FE900800EE4F604F
:100EAB000FE02AFA74003BFBA31FBFFFF01E80ED7F
:100EBB007E0F901500E02AFA74003BFBA3DEF67E52
:100ECB000F90150FE02AFA74003BFBA3DEF67E2091
:100EDB00901546E02AFA74003BFBA3DEF690000166
:100EEB00EAF0A3EBF022900000E004B4FE08745586
:100EFB00121488020F8FF014F5F07408A42410F864
:100F0B00E5F03400F5A07A04901401E0F2121D39DB
:100F1B00DAF9E0B4FE0E900000E014F074551214F0
:100F2B0088020F8FFDA3E0FCA3A982AA8390000384
:100F3B00E02CF0A3E03400F0900005E0F5F0F212A5
:100F4B001D39E0F2FB121D39ECF2121D39EDF212D4
:100F5B001D3974FFF2121D39F2121D39F2121D39AF
:100F6B00F28A838982A9F0E08BA0F3A309B900016F
:100F7B000BDCF4900005E9F0A3EBF0C226C225745C
:100F8B00AA121488C22322202606202503120AE463
:100F9B0074AA121488C22322121CAE74AA121488CB
:100FAB00C22320340B901522E04402F090E000F0B5
:100FBB00D297D29622121ADD121EF174AA1214883D
:100FCB00C22322901401E0B4400040028013B40A03
:100FDB0000400E900007F0121CAE74AA1214888009
:100FEB00057455121488C22322901401E0B40A0030
:100FFB0040028022FA780075A015F2121D39E0B478
:10100B003F005012B43200400DF2DAEF74AA121402
:10101B0088121CAE800A901500E4F07455121488E7
:10102B00C22322780175A0149015467D20E2F012A0
:10103B001D39DDF9121CAE121EF174AA121488C2EE
:10104B00232290155CE0547FF56A901401E054075D
:10105B00F568901402E0B41B004002741AF569C2E3
:10106B002322900009E075F01E700375F018B4018F
:10107B000375F019901401E0B418004001E49015C9
:10108B0085F0901402E0B43C004001E4901586F02A
:10109B00901403E0B43C004001E4901587F09014E9
:1010AB0004E0B5F0004001E4901588F0D23DC22376
:1010BB0022901401E0700575F0188060B40105757D
:1010CB00F0198058B4020575F01E8050B4030575F5
:1010DB00F01E8048B4040575F01E80407402900029
:1010EB0009F090150F7400F0A37400F0A37400F0D6
:1010FB00A37400F0A37418F0A37400F0A37400F0B1
:10110B00A37400F0A37400F0A37400F0A37400F0B8
:10111B00A37400F07455121488021218900009F091
:10112B00901402E0B4180050B390150FF0F55590E1
:10113B001517F0901403E0B43C0050A0901510F07C
:10114B00F556901518F0901404E0B43C00508D90B7
:10115B001511F0F557901519F0901405E0B5F00046
:10116B0040030210E7901512F0F55890151AF0C2D3
:10117B0023901406E0B41804D22380054003021018
:10118B00E7901513F0F530901407E0B43C004003E2
:10119B000210E730230560030210E7901514F0F5F9
:1011AB0031901408E0B43C0040030210E7302305F3
:1011BB0060030210E7901515F0F532901409E0B5B5
:1011CB00F00040030210E730230560030210E790A4
:1011DB001516F0F53390140AE0A2E09222A2E192E8
:1011EB0005A2E2921FA2E3922AA2E4922BA2E5921D
:1011FB002DA2E6922EA2E79213900008F0D2962031
:10120B002204C2018002D20174AA121488121CAEED
:10121B00121EF1121E8CC22322900009E075F01EE3
:10122B00700375F018B4010375F019901401E0B454
:10123B00180040028047901402E0B43C004002804A
:10124B003C901403E0B43C0040028031901404E065
:10125B00B5F0004002802690151AF0901403E09030
:10126B001519F0901402E0901518F0901401E0900D
:10127B001517F074AA121488121CAE80057455123F
:10128B001488C22322901401E0FBA3E0FA901522EC
:10129B00E04AF0FAA3E04BF090E800F090E000EAAF
:1012AB00F074AA121488C22322901401E0F4FBA359
:1012BB00E0F4FA901522E05AF0FAA3E05BF090E824
:1012CB0000F090E000EAF074AA121488C223229076
:1012DB00E800E0FB90E000E0FA74AA121488EB122D
:1012EB001488EA121488C22322D201D29174AA1252
:1012FB001488C22322D29120151720001CC23F3024
:10130B002217301F14300304D201801A12193880AF
:10131B0008103F028003121938C201C200C21574B3
:10132B00AA121488C22322202B02D20074AA1214F0
:10133B0088C22322302206C2AFD215D2AF74AA12B2
:10134B001488C22322901401E0A2E0900008E092DE
:10135B00E35000F075A015781B901402E0F9F20829
:10136B00A3E0FAF208A3E0F2FBC3740099748D9A20
:10137B0074279B400302139C900008E054F7F090F5
:10138B00151B7400F0A3F0A3F0745512148802130C
:10139B00A4121CAE74AA121488C22322900000E07F
:1013AB00FFFA1214889000100FDF02804EE0121427
:1013BB00882AFAA3E01214882AFAA3E01214882AC6
:1013CB00FAA3E01214882AFAA3E0FDA3E0FEA3E03F
:1013DB00FCA3E0A31214882AFAEC1214882AFAC090
:1013EB0082C0838D828E830CDC028009E01214880C
:1013FB002AFAA380F3D083D08280AEEA121488C27B
:10140B0023227F037E007A00903400E01214882A96
:10141B00FAA3DEF7DFF59020007E10E01214882A85
:10142B00FAA3DEF7EA121488C223229015657F20F7
:10143B00E4F0A3DFFC756600C234C235C2369015EA
:10144B0022E04402F090E000F074AA121488C22348
:10145B0022E430350244013036024402FA12148879
:10146B009015657F20E01214882AFAA3DFF7EA12A1
:10147B001488C2232274AA121488C22322C0E0C08B
:10148B0082C08375831F855C82F0E55C04F583B5B0
:10149B005B072020FAD29980F685835C202002D24C
:1014AB0099D083D082D0E02275A891C28CC28EC213
:1014BB008F902D4712022A902D5712022A902D7FC2
:1014CB0012022AC20BC20DC212C20FC20CC210C230
:1014DB000EC207851211758A00754C00752940756F
:1014EB002A017555007556007557007558007533F0
:1014FB000090151BE0F530A3E0F531A3E0F532C207
:10150B00AF75B80675A81FD246D28CD2AFC22312C4
:10151B001AB512050430230D75A891C28CC28E1218
:10152B000BB90216FA100C183004E7C2041202C7EA
:10153B001207DB3001DC75A891C28CC28E0216FA41
:10154B00E539540375F00AA4F8E538540F28200E3A
:10155B0009B415BED20E7A0080B8F890156EEA5415
:10156B000323738006800A800E8028B8166F0A80CA
:10157B00A1B817690A809BB818030A8095B8005D5B
:10158B0075461875127875295BC206902DCF12021D
:10159B002A804FB8193175461E751296752915C2DA
:1015AB0006E53930E20AD206902DEA12022A803281
:1015BB00900009E0B40208902DE112022A802390DA
:1015CB002DF312022A801BB8001375461975127D74
:1015DB0075294DC206902DD812022A8005C20E0223
:1015EB00151D902D6512022AC2AF854341854442D9
:1015FB00D2AFE54175F014A4F541A8F0E54275F0C2
:10160B0014A428F542754E00754D00D210D20FE58B
:10161B0039540375F00AA4F5F0E538540F25F0049E
:10162B00F548F554E53B540775F00AA4F5F0E53A97
:10163B00540F25F0F549F553E53D540775F00AA411
:10164B00F5F0E53C540F25F0F54AF552E53F540310
:10165B0075F00AA4F5F0E53E540F25F0F54BF55166
:10166B00D23A121AB5C202C218C21912050430239B
:10167B000302152320100D75A891C28CC28E7528FC
:10168B00000216FA301902C219301836C2181207A6
:10169B00DB30010975A891C28CC28E8052300D0BC4
:1016AB001209C6902D6512022A8017902D72120214
:1016BB002AD296E511600BD51108D236C201C2228F
:1016CB00802D30021AC202301603120A0F301B0390
:1016DB00120A82120847121F7A1202C712024E30E8
:1016EB00170AC217301605C216120A4002167612D6
:1016FB001AB5D297D296901522E04409F090E000EB
:10170B00F002012375A891C28CC28EC215C23FC2D2
:10171B001AC218901522E054FEF090E000F0902DC4
:10172B004F12022A12193820426420413A204025D8
:10173B00754618754000901554E0B4E90C902DCF08
:10174B0012022A9015540217AC902DC612022A9041
:10175B0015540217AC902DD812022A9015567546C7
:10176B00197540000217AC304012902DE112022A7D
:10177B0090155A75461E7540000217AC902DEA1253
:10178B00022A90155875461E7540040217AC902D11
:10179B00F312022A90155875461E754000C240C2BE
:1017AB0041E0A3750F00F50EE0F50D7547007509C7
:1017BB0036750C00750B0A750A01D209850E4F128E
:1017CB001AB5C2AF75B802850E8A202E13902D9FC5
:1017DB00202703902D9212022A75A81BD28C8057BA
:1017EB0075A81FC28B902D5712022A902DB9120289
:1017FB002A20412F204016902DC612022A74EA751A
:10180B000F00F50E850E4F74C2F50D802A902DD862
:10181B0012022A750F0074E0F50E850E4F7497F5C2
:10182B000D801474BA750F00F50E850E4F74F0F51C
:10183B000D902DF312022AC246C28DC28FD2AFC2B7
:10184B00231224C9D203120504302306120BB9202C
:10185B000167302714901589E0B4050C902D921276
:10186B00022AD297C2278001F030240FE545B4033A
:10187B0002800875450312251B80CB300216754577
:10188B000012251BC224C2021208477545011225FE
:10189B001B12024E30181C75450212251BC2181262
:1018AB0007DB121F7A20011130150B902DAC1202A1
:1018BB002A801202185102185175A891C28CC28E3F
:1018CB007528008056120504202330300225C202F1
:1018DB001202C71207DB200136201517D292202ED9
:1018EB0009902D9212022A021851902DB912022A38
:1018FB000218513018CFC2180218D0120BB930157C
:10190B00DBD29175A891C28CC28E752800800CD247
:10191B009175A891C28CC28E752800901522E04457
:10192B0001F090E000F0D296C203020123121AB527
:10193B0090150FE0F555A3E0F556A3E0F557A3E09E
:10194B00F558A3E0F530A3E0F531A3E0F532A3E0C1
:10195B00F533A330000390150FE0F54BA3E0F54AE8
:10196B00A3E0F549A3E0F548303D12901585E0F56D
:10197B004BA3E0F54AA3E0F549A3E0F54890000935
:10198B00E070087528007567048027B40108752876
:10199B0001756704801CB403087528047567018002
:1019AB0011B4040875280275670180067528037544
:1019BB0067017536FC7537BFE54875F00A8485F00D
:1019CB00384540F539E54975F00A8485F03AF53B21
:1019DB00E54A75F00A8485F03CF53DE54B75F00A58
:1019EB008485F03EF53F2290400374C2C2AFF09065
:1019FB004000E0E0F4FCE0F4FD9040037436F0901E
:101A0B004000E4F0F0D2AF202C43ED13547FFDECFB
:101A1B00132403FCED3400FDC3E5349CFC90600300
:101A2B00F0E5359DFD906003F075F00030E7037530
:101A3B00F0FFAEF0C390155EE03CFCF0A3E03DFD83
:101A4B00F0A3E03EFEF020E70C4D4C702EC22CAD07
:101A5B002CAC2D804775F00AF47013EDF4700FEC7D
:101A6B00F4B45000500803030303540FF5F0E52CB6
:101A7B00C395F0FDE52D9400FC802175F00AEE7006
:101A8B0011ED700EECB45000500803030303540F18
:101A9B00F5F0E52C25F0FDE52D3400FC75A0407824
:101AAB0001EDC2AFF2ECF2D2AF22D22CE490155E74
:101ABB00F0A3F0A3F0AD2CAC2D121AA7227A108054
:101ACB0003121D39E2F0DAF9FAE0C39A70FB121D2A
:101ADB003922120D02121C65903440E0B4550D9062
:101AEB002000E0FCB4FE004006021B8A021BDD90C6
:101AFB002003E0A3F8C3740098E0F8740C9850032B
:101B0B00021B8A90200075A0007800ECF27D00FE8D
:101B1B00121D39E0FBF2121D39E0FAF2121D397F6A
:101B2B000DE0F22CFC74003DFD121D39DFF3BE00FD
:101B3B0004D226804AC226902010781075A0007F10
:101B4B0008E0F22CFC74003DFD121D39DFF3DEEFD3
:101B5B007E08E0F2121D39DEF9900003E0FFA3E0EE
:101B6B00FE90280075A0087800EE4F6012E0F2128C
:101B7B001D392CFC74003DFD1FBFFFED1E80EA7F5D
:101B8B000F780075A015903400E0F2121D392CFC73
:101B9B0074003DFDDFF37F0F780F75A015903410A7
:101BAB00E0F2121D392CFC74003DFDDFF37F207831
:101BBB004675A015903420E0F2121D392CFC7400F0
:101BCB003DFDDFF3ED8AF0B5F008EC8BF0B5F002DC
:101BDB008030901522E054FDF090E000F0D235C239
:101BEB0097C296122CB8122CB8D297D2967C209012
:101BFB0034FF7A107400A3F0DAFCE0B400FCDCF2E2
:101C0B008010900000E06006C226D2258004D22608
:101C1B00C2257D04785590150FE0F6A308DDFA7DFB
:101C2B00047830901513E0F6A308DDFA900008E075
:101C3B00A2E09222A2E19205A2E2921FA2E3922AD3
:101C4B00A2E4922BA2E5922DA2E6922EA2E792138A
:101C5B00202204C2018002D20122902CE175A00047
:101C6B0078007A10E493F2121D39DAF8902CF175A2
:101C7B00A01578007A0FE493F2121D39DAF8902D43
:101C8B001275A015780F7A0FE493F2121D39DAF85A
:101C9B00902CFC75A01578467A16E493F2121D3938
:101CAB00DAF822202606202503120AE4120E6C789D
:101CBB000075A000902000E2FC121AC8EC70030221
:101CCB001D02C31304FC121AC8DCFB900003E0FCDA
:101CDB00FFA3E0FD7A04EDC313FDEC13FCDAF7EF81
:101CEB00540F60010CBC0002800D780075A00890A9
:101CFB002800121AC8DCFB780075A015903400126E
:101D0B001AC8780F75A015903410121AC87846753A
:101D1B00A015903420121AC8785675A0159034303F
:101D2B00121AC89034407455F0E0B455FC22A30845
:101D3B00B8000205A022901537E0540F2323901D05
:101D4B004D73021D8D00021D8D00021D8D00021DA5
:101D5B008D00021D8E00021D9A00021DA600021DA1
:101D6B00B200021E1B00021E3500021E4F00021E97
:101D7B006A00021D8D00021D8D00021D8D00021DCB
:101D8B008D0022901538E0543FFA7918021DBE9051
:101D9B001538E0543FFA7919021DBE901538E054FE
:101DAB003FFA791A021DBE901538E0543FFA791BA1
:101DBB00021DBEE562C39561F4B40500500280F3C9
:101DCB0075831C75A01B85628274FF4480FBF074C5
:101DDB0001A882F205827400F02BFB7400A882F23A
:101DEB000582E9547FF02BFB7400A882F20582EA8E
:101DFB00F02BFB7400A882F20582EB03547FF07486
:101E0B0001A882F205828582629060057406F02239
:101E1B00901537E0232354C0F9A3E0543F49F990C0
:101E2B001522E049F090E000F022901537E02323D3
:101E3B0054C0F9A3E0543F49F9901523E049F090C1
:101E4B00E800F022901537E0232354C0F9A3E054A7
:101E5B003F49F4F9901522E059F090E000F0229000
:101E6B001537E0232354C0F9A3E0543F49F4F9900C
:101E7B001523E059F090E800F022E55EC3955DF480
:101E8B00229060027415F0906000741BF07407F0E0
:101E9B00A374BBF09060047408F09060027405F0BA
:101EAB0090600274B5F09060057406F09080027437
:101EBB0015F0908000202D04741B80027413F074B5
:101ECB0007F0A3202D0474BB800274CCF090800427
:101EDB007408F09080027405F090800274B5F09055
:101EEB0080057406F022121AB5901546E0F52B60AA
:101EFB0000A3A3A3E0F52DA3E0C0E054FEC39432EE
:101F0B00F52CE52D9400F52D9040037476F0904060
:101F1B00017F32E52C2402F52CF0E52D3400F52D54
:101F2B00F0122CD8DFED7F19E52CC39402F52CF0C1
:101F3B00E52D9400F52DF0122CD8DFECD0E0F52C2C
:101F4B00F0E52DF0121F5322900009E0B40005902C
:101F5B00154C8013B4010590154E800BB4020590FF
:101F6B0015528003901550E0F535A3E0F53422C0EF
:101F7B00D0C0E0C0F0C082C083202D0E30130BE523
:101F8B0062C39562F4B40800500302202B75831CC6
:101F9B0085628274FEF0F5F075831B7401F0058287
:101FAB0075831C7400F025F0F5F075831BE4F005C8
:101FBB008275831C7460F025F0F5F075831BE4F0DB
:101FCB00058275831CE54BF025F0F5F075831BE45A
:101FDB00F0058275831CE54AF025F0F5F075831B3F
:101FEB00E4F0058275831CE549F025F0F5F0758367
:101FFB001BE4F0058275831CE548F025F0F5F075C0
:10200B00831BE4F0058275831CE5F003547FF075A8
:10201B00831B7401F005828582629060057406F063
:10202B00D083D082D0F0D0E0D0D022204603D28C07
:10203B0032C0D0C0E0D214300D02B2967402C28C02
:10204B00C58AD28CF54FE4C54C308D0704700274F1
:10205B0003C28DF550C3E54F948AE5509400401BA5
:10206B00C3E529954FE52A95504004D20880137497
:10207B00B5954F74029550C2085007C20BC20D02A2
:10208B00215130080D30070A200A28C207054702E4
:10209B002151200B6BA208E53713F537E53613F505
:1020AB0036B4FC78E537B4BF73300807D20AD207D1
:1020BB00022151C294D2177400B54808B54905B531
:1020CB004A028016E53F540775F00AA4F5F0E53E89
:1020DB00540F25F0F54BF551D23A750938750B08AD
:1020EB00750A08754700D20BC20AC207300F577525
:1020FB004500754E00754D00D28ED28FC20F8046B3
:10210B00C000A208A809E613F6D000D50A0E0509EF
:10211B00750A08D50B06C20BD20DD20C300804D2AF
:10212B000780230547C207E54354F02544C4F50F48
:10213B00E54F54F02550C4254350020544C3950F79
:10214B00F54350021544D0E0D0D032204603022193
:10215B006CC0E0054CE54C7005D204754C03D0E027
:10216B0032C0D0C0E0C0F0C082C08330091130153E
:10217B0007300504D2968002B296C20702221DC018
:10218B0000A809E630E00E301507300504D2968022
:10219B0002B296D20703F6D0000547E50AC333F522
:1021AB000A506F750A010509D50B67750936750B52
:1021BB000A754700854854854953854A52854B51CA
:1021CB00D23AE54875F00A8485F0384540F539E593
:1021DB004975F00A8485F03AF53BE54A75F00A84B7
:1021EB0085F03CF53DE54B75F00A8485F03EF53FF7
:1021FB00D28F302E1DD5671AB209050CC28C758A89
:10220B00FE756701E5285407B40200503B7567045F
:10221B008036B209850E4FE50CC3950D4002054F74
:10222B00050CC28CE4C3954F258AF58AD28C201AF3
:10223B000DE509B43B12D21AD218D294800A20248D
:10224B0007E509B43E02D224D083D082D0F0D0E08F
:10225B00D0D0322046030225F7C0D0C0E0E54E6057
:10226B0004154E8019E54D601AC3E4954D754D006C
:10227B00C28E258C5004D28E8009F58CD28ED0E084
:10228B00D0D03212251BC21AE5457007200D0DC2A6
:10229B00948009B40206D21AD294D218C0F0C0832B
:1022AB00C082200D030223E8201A0C101406C20D65
:1022BB00C20BD20F0223E853A8FB854C17858A1655
:1022CB00E547A20785441485431543A8049211F5ED
:1022DB00F0B428004003022366C3742895F023F55D
:1022EB00139415400BC20DC212C20BD20F0223E87E
:1022FB00E514C313C51513F51420110BC39516E57F
:10230B00159517400280021513E5148513F0A4F5FB
:10231B001685F017E5158513F0A42517C313C516FD
:10232B0013C516C313F517E51613F516E517C313E7
:10233B00F515E51613C515C313C51513F51425416E
:10234B00F541E5153542F542E5162541F54DE51705
:10235B003542F54E154ED2120223F0942823F51375
:10236B009415400BC20DC212C20BD20F0223E8E52B
:10237B0014C313C51513F51420110BC39516E515CE
:10238B009517400280020513E5148513F0A4F5168A
:10239B0085F017E5158513F0A42517C313C5161380
:1023AB00C516C313F517E51613F516E517C313F585
:1023BB0015E51613C515C313C51513F514C3E54160
:1023CB009514F541E5429515F542C3E5419516F592
:1023DB004DE5429517F54E154ED212800885424EAB
:1023EB0085414D154EE545B403028008B40102D278
:1023FB00190224B9300D5C301259C297901522E0A6
:10240B0054F6F090E000F0851211E539540375F0A5
:10241B000AA4F5F0E538540F25F0F548E53B5407D1
:10242B0075F00AA4F5F0E53A540F25F0F549E53DB2
:10243B00540775F00AA4F5F0E53C540F25F0F54A66
:10244B00805C7400B5481CB54919B54A160548059A
:10245B004B804BD297901522E04408F090E000F0AF
:10246B00121AB50548E548B546347548000549E5E7
:10247B0049B43C2A754900054A300610E54A75F007
:10248B000A84E5F0600674022548F548E54AB43C39
:10249B000D754A00054BE54BB41803754B00854889
:1024AB0054854953854A52854B51D202D23A054540
:1024BB00534503D082D083D0F0D0E0D0D032302D32
:1024CB004E30134B74F0122907747F122907747F57
:1024DB0012290774011229077401122907900009A8
:1024EB00E0B400028010B4010474208009B402042B
:1024FB00746080027440454B122907E54A12290784
:10250B00E549122907E54812290774F71229072212
:10251B00302D1930131620375CE545B4001174F1DA
:10252B00122907E548540F44001229070225F6B477
:10253B00011574F1122907E54854F075F010844425
:10254B00101229070225F6B4021174F1122907E5BE
:10255B0049540F44201229070225F6B4031474F1D1
:10256B00122907E54954F075F010844430122907FD
:10257B00D2370225F6E545B4001174F1122907E5AF
:10258B004A540F44401229070225F6B4011574F181
:10259B00122907E54A54F075F010844450122907AC
:1025AB000225F6B4021174F1122907E54B540F44BE
:1025BB00601229070225F6B4033174F1122907E5DD
:1025CB004B54F075F01084F5F0900009E0B4000264
:1025DB008010B4010474028009B4020474068002F2
:1025EB00740445F04470122907C23722C0D0C0E0F2
:1025FB00C0F0C083C08230150302269E203D43905D
:10260B001589E004F00548E548B5464D75480005C9
:10261B0049E549B43C43754900054A304110204017
:10262B000DE54A75F00A84C5F06003754802E54A6A
:10263B00B43C26754A00054BE54BB4181C754B0092
:10264B008017901585E0F54BA3E0F54AA3E0F5491B
:10265B00A3E0F548C23D20273AE54BB53035E54AB6
:10266B00B53130E549B5322BE548B53326D291303B
:10267B002B0D200506D215D23F8018D201801430C5
:10268B0000052005F680EE85554B85564A85574942
:10269B00855848D202C21AC294901522E04401F028
:1026AB0090E000F0D082D083D0F0D0E0D0D032E5F3
:1026BB0060C3955F855F1BB4070050030229BD12F1
:1026CB002B31B4F1030229C1B4F06B122B3120E78B
:1026DB0063B47F62122B3120E75AB47F02800B2444
:1026EB0009F5F0900007E0B5F04C122B3120E744D0
:1026FB00B402028006B4013E022805122B3120E7FA
:10270B0033B410028008B430028003B47F28122B3C
:10271B003120E720F51AB415030228A2B4160302E0
:10272B0028A2B417030228A2B418030228A2B419D2
:10273B0005022744151B0229B7E560C3955FB41248
:10274B000050030229BD122B3120E7E8C3943075EA
:10275B00F00AA4F5F0122B3120E7D9C3943025F001
:10276B00B418004001E4901585F0122B3120E7C41A
:10277B00B400C3122B3120E7BBC3943075F00AA40D
:10278B00F5F0122B3120E7ACC3943025F0B43C00AC
:10279B004001E4901586F0122B3120E797B4009698
:1027AB00122B3120E78EC3943075F00AA4F5F0128A
:1027BB002B3120E73FC3943025F0B43C004001E4BB
:1027CB00901587F0122B3120E72AB4002A122B31F7
:1027DB0020E721C3943075F00AA4F5F0122B3120B9
:1027EB00E712C3943025F0B41F004001E490158824
:1027FB00F00228A202273F022741E560C3955FB490
:10280B000A0050030229BD122B3120E7E7C3B401A4
:10281B00E6122B3120E7DDC3F5F0540FB41800405E
:10282B000302289F901585F0E5F0546075F0208425
:10283B00900009B4000474018010B4010474028088
:10284B0009B40204740380027402122B3120E74195
:10285B00C3B43C00400302289F901586F0122B3125
:10286B0020E72EC3B43C00400302289F901587F04D
:10287B00122B3120E71BC3B41F00400302289F908B
:10288B001588F0122B3130E70BB4F705D23D022936
:10289B00B702273F022741122B3130E72CB4F72C1C
:1028AB00E51AB4152AD291C201201510200017C2C7
:1028BB003F302212301F0F121938800A103F02804E
:1028CB0005121938C20002292D0229B702273FB47D
:1028DB00160C3022F1C2AFD215D2AF02292DB4178C
:1028EB0005D20102292DB41808202B02D20002298F
:1028FB002DB41905D23D02292D0229B7C0E07583ED
:10290B0018855E82F07400758317F00582E55D65AE
:10291B0082600385825E9080057406F0851B5FD014
:10292B00E02274F0758318855E82F074007583174E
:10293B00F00582E55D6582607385825E747F7583C9
:10294B0018855E82F07400758317F00582E55D656E
:10295B0082605985825E7403758318855E82F0747C
:10296B0000758317F00582E55D6582603F85825EA9
:10297B007402758318855E82F07400758317F005F9
:10298B0082E55D6582602585825E74F775831885A7
:10299B005E82F07400758317F00582E55D658260D9
:1029AB000B85825E9080057406F08000851B5F02AC
:1029BB0026BA2202273F122B3120E7F7C0E054F052
:1029CB0075F01084540FB40018D0E0540FF5F0904C
:1029DB00000AE054F045F0F090000EE014F00229EC
:1029EB00B7B40116D0E0540F75F010A4F5F09000B9
:1029FB000AE0540F45F0F00229B7B40212D0E054AC
:102A0B000FF5F090000BE054F045F0F00229B7B44D
:102A1B000316D0E0540F75F010A4F5F090000BE006
:102A2B00540F45F0F00229B7B40412D0E0540FF55F
:102A3B00F090000CE054F045F0F00229B7B4051605
:102A4B00D0E0540F75F010A4F5F090000CE0540F8B
:102A5B0045F0F00229B7B40612D0E0540FF5F09010
:102A6B00000DE054F045F0F00229B7B4075DD0E05B
:102A7B00C0E0540175F010A4F5F090000DE0540F78
:102A8B0045F0F0D0E0546075F02084900009B4005C
:102A9B000990000EE004F0022AE1B4010990000E47
:102AAB00E004F0022AE1B4020B740390000EE00480
:102ABB00F0022AE1B4030B740290000EE004F00262
:102ACB002AE190000EE004F0022AE1D0E090000E23
:102ADB00E0E4F00229B790000EE0B4004490000D42
:102AEB00E0901585F090000CE0901586F090000BAF
:102AFB00E0901587F090000AE0901588F090000F99
:102B0B00E0E4F0D23D901589E4F020011120270E6E
:102B1B00D227C23FC215902D9F12022AC2970229BB
:102B2B00B7E4F00229B7758316851B82E0051B22DB
:102B3B00C0D0C0E0C082C08310990C109826D083FF
:102B4B00D082D0E0D0D032C299E55B655C7005C213
:102B5B0020022B6CD220855B82055B75831FE0F511
:102B6B0099022B43E59975831E855A82F075831D57
:102B7B00209A04740080027401F0A3E55965826009
:102B8B000385825A022B43C0D0C0E0C082C0839021
:102B9B008005E030E103022C41908005E030E20338
:102BAB00022C8C906005E030E103022BCD90600588
:102BBB00E030E205022C1580D6D083D082D0E0D055
:102BCB00D032E5616562700F9060057404F090601F
:102BDB000274B5F0022BB890600274A5F0906002FD
:102BEB007415F075831B856182E06008906000743A
:102BFB001FF08006906000741BF075831C8561824A
:102C0B00E0906003F00561022BB8906001E07583E2
:102C1B001985648220E504740080027401F09060D1
:102C2B0003E075831A856482F0A3E5636582600314
:102C3B00858264022BC2E55D655E700F9080057422
:102C4B0004F090800274B5F0022BA490800274A55E
:102C5B00F0202D1D9080027415F0758317855D8211
:102C6B00E06008908000741FF08006908000741B59
:102C7B00F0758318855D82E0908003F0055D022B73
:102C8B00A4908001E075831785608220E5047400B1
:102C9B0080027401F0908003E0758316856082F0EA
:102CAB00A3E55F65826003858260022BAE7A3EEA04
:102CBB00C0E0122CC6D0E0FADAF5227A007B20DADB
:102CCB00FEDBFC227A007B0ADAFEDBFC227A007B3D
:102CDB0032DAFEDBFC22000000000000080A0202D0
:102CEB0000000000000000000000000000000000D9
:102CFB000000000100040047C744E8397B396CEE43
:102D0B0000E5CDBECEBD00000000001800000000A5
:102D1B00000000008D27010120534D505445204DDC
:102D2B00616368696E652020000201202056657280
:102D3B0073696F6E20312E363920200001015265E8
:102D4B0061642000010147656E20200001062D2DD6
:102D5B003A2D2D3A2D2D2E2D2D0002014C6F636B2C
:102D6B0065642020202000020153656C66204765B6
:102D7B006E20200002014177616974696E672053F0
:102D8B004D505445202000020152756E6E696E67DE
:102D9B002020200002014D544320536C61766520A6
:102DAB0000020149646C696E67202020200002013B
:102DBB00562D53796E632020202000020B32332EC8
:102DCB0039373600020B32342066707300020B3237
:102DDB00352066707300020B33302066707300026F
:102DEB000B32392E39376400020B32392E39376EDC
:012DFB0000D7
:00000001FF
